:020000040000FA
:10000000830A7F0EE2018008810882088208830843
:100010008308830883088408840884088408840883
:10002000840884088408850885088508850885086B
:100030008508850885088508850885088508850858
:100040008508850885088608860886088608860843
:100050008608860886088608860886088608860830
:100060008608860886088608860886088608860820
:100070008608860886088608860886088608860810
:1000800086088608860897089708970897089708AB
:100090009708970897089708970897089708970868
:1000A0009708970897089708970897089708970858
:1000B0009708970897089708970897089708970848
:1000C000970897089708A708A708A708A708A708E8
:1000D000A708A708A708A708A708A708A708A708A8
:1000E000A708A708A708B708B708B708B708B70848
:1000F000B708B708B708C708C708C708C708D708A8
:10010000D708E708F70825006300170C0200070569
:1001100067044704C70505040B0C060069006A0064
:100120006B00460427050107930A2902430646058A
:100130000106980A460421024307930A080243066F
:100140008E0A01092A00E806AA030F0C6A01A90217
:1001500009028A000307690048024307900AAB02BC
:100160004307910A67004604060203000000830A61
:0203FE00180CD9
:021FFE001800C9
:00000001FF
